:020000040000FA
:02000000E02FEF
:08000800F000030EF100831269
:100010000313F21D59287608F90B1628FF3E8100BC
:100020007708242086007808F9001A2881007708CC
:1000300024208600770A1F39F700FA0A0B11710E87
:100040008300F00E700E090082074B3449344334AC
:1000500041340B3409340334033403340334093496
:100060000B344134433449344B34833489348B3436
:10007000C134C334C934CB34CB34CB34CB34C9349E
:10008000C334C1348B34893483348207013402345D
:100090008207303431343234333434343534363406
:1000A00037343834393441344234433444344534B9
:1000B0004634831203130B185E281F28060800001D
:1000C0000B102D300102031C6828721381011F28B8
:1000D000721781011F28F21E7428F2122108F600FF
:1000E0002308F900F8007A28F2162008F600220802
:1000F000F900F800080083160313C0308100831252
:1001000003130A30AC007A21F21C8828AC0B832838
:100110000614F7016B2000308A00F2150B118B16C4
:100120000800C830A000E530A1000130A200013075
:10013000A300F401F501F201F30178270030A124B6
:100140000130A124FF306D06031D0800EC01ED0114
:10015000AB2608000630831603139C001F309B005B
:10016000F730850034308600831203138501860141
:10017000CC20313090000F3092000B178B17031AF0
:10018000C5280E30CC231A30CC2383120317173026
:1001900085008312031308008316031318114030DF
:1001A0009900981683120313981718160800EC1973
:1001B000DA2822296C1F22296D1C2229731D0A2985
:1001C00018160D24F31922292408243A0319E928C2
:1001D000E128C824F31922296927AC00ED1EF22872
:1001E0007930F9286D1FF6287630F928ED1F22297D
:1001F00066302C06031DE1281812242124308221A8
:10020000F310B201EA24240882210D302406031DD4
:1002100002292029ED1C222924216430A800280865
:10022000831203178D00831603170C148312031710
:100230000C0883120313031920298221A80A0F290D
:100240006D21C02174100800ED1D2829F3212A29F1
:100250007B205F2145308400F2134721F2133E30AA
:100260008400453068060319402947214C3084003A
:1002700068060319402947210730840704083829F4
:10028000F217472103308221F03082210800073025
:10029000BB000008AC0001303B06031D58290310C9
:1002A000AC0DF21B2C142C088221063084020800AD
:1002B0000310AC0D2C088221840ABB034929FF30AE
:1002C000B500B60081308316031392008312031326
:1002D00091018C106B089E210800FF303506AC00A0
:1002E000FF30360682212C08822102309E218C1C90
:1002F00077290800F21006080B10143051220B1851
:10030000F2140800B3006400ED199B290830B00016
:10031000330CAC21B30C031C97297212AF0AB9211C
:100320002F08053A03199729B00B88290800AF0157
:100330007216B92194293308E9210800AA00063071
:10034000B0007216B9217212B921B00BA32972162E
:10035000B921AA0B9F29080001300318B606031023
:10036000B50CB60C031C08000830B6068430B50680
:10037000080064008C1CB9298C10721A6B200800CC
:100380008B12000006100800721BCA293D1CCE29E2
:10039000BD0ADA293D18CE29BD0ADA298C1CC429E8
:1003A00081308316031392008312031391018C1082
:1003B00003140800C2308316031392008312031340
:1003C00091018C10031008000C1EE42999006400B0
:1003D00008008A242030E421FB0A0F307B05031D2E
:1003E0000800F6210800FB01F62108000D30E42189
:1003F0000A30E42108003208FF3C031C0800AD0A63
:10040000052A3208FF3C031C08001C2272190B2A23
:1004100037088000080037088317800083137211A3
:100420000800AD031C227219172A00080800831760
:10043000000883137211080072113208013C03187E
:100440002A2A32083F3C03182E2A32089F3C031800
:10045000352A3D2A32086E3E840008003208AC007E
:1004600002302C02A03E840008003208AC0040306C
:100470002C02103E8400721508003208AC00A03037
:100480002C02903E840072150800FA30A90000008A
:10049000A90B472A0800AA00C8305122AA0B4C2AEF
:1004A0000800A80045224522452245224522A80BE6
:1004B000522A0800FB21B20A0830B000B70CAC2168
:1004C000B00B5E2A08000630B1001122AC00031008
:1004D000AC0C2C08203A03196F2A2C08E421B20A2C
:1004E000B10B652A1122B900B90C0F30B9050319F7
:1004F000852A2D30E4210A303902031C822AB900F2
:100500003130E4213908303EE42129083206031D48
:100510008B2A2A30E4210800F2118B128316031370
:1005200084308100831203130B108B152830840054
:10053000FB237210FF30B500B6009101C23091006C
:100540008C10B9270318F02AC421B40C34087E3A61
:10055000031DA12AB4010830B000C421031CB92A2C
:10056000AF0AB40C2F08053A0319BB2AB00BAD2A09
:10057000CF2AAF01B12AC4210318C02AAF01B62A7D
:10058000C4210318962A3008033A031D962AAF01A6
:10059000721CAA2A2E080F3C0318962ADF2A721C06
:1005A0007214AE0A2E08FF3A0319962A2E08023C4E
:1005B000031C5A223808B7003408B800AA2AEC18DD
:1005C000EC2AFF30B606B50637083606031D962A14
:1005D00038083506031D962A0230AE027517F51647
:1005E0008B11080075136C1A082B6C1D08006C1F0A
:1005F0000800B2013E308400B223031C002B082BFC
:10060000EC1F0800B20161308400B223031C080013
:100610006D1A4B2BFF30A9000D30B2001222B90029
:100620003918152B0730B2070E2B3208A8000D30F1
:1006300032060319242BB91B222B0730B2021222D7
:10064000B900172B3208A9000730B20063223E30F0
:10065000E421B201632228080D3A031D322B0D302C
:10066000B2003F2B2C30E4210E30B2006322280868
:10067000320603193F2B2C30E421B20A362B3A30D4
:10068000E4210230B207AD022D080319542BB20A3F
:100690001122E421442BB201F3212D080319542B1C
:1006A0001122B20AE9214D2B0D30E4210A30E42158
:1006B0000800F512EC1E08006C1F08002D08BA0097
:1006C0000D30B2001222B9003918B02B1430B2002C
:1006D0001222B900B91F742B391808000730B2076D
:1006E000443C031C0800682B0630B2023208A80004
:1006F0003E308400B223031C7E2BA02BEC1F08008D
:100700002808B20061308400B223031C08002808C6
:10071000B2000730BB003E3084000008BC0003106C
:100720003C0DB7000408A90012220139B7040122C8
:1007300029088400BB0B9D2BA02BB20A840A8D2BA9
:100740002808063EB20012228038B70001227B2022
:100750005F21B20112228221B20ABA0BAA2B6D21AB
:10076000C02108000730BB000008BC000408AB0033
:100770000310BC0D1222B400341034083C06031DD3
:10078000CA2B2B088400BB0BC72B03140800B20A2A
:10079000840AB42B03100800A800831203170B303F
:1007A0008F002C308D00831203132808332726274F
:1007B000831203178D000E088F0083120313262760
:1007C000AC00003A031908002C08E421013033275B
:1007D000DF2B8312031708308F0029308D0083121E
:1007E00003132627AC00003A031908002C08E42163
:1007F00001303327F12B80013D3004060319080036
:10080000840AFB2BB2018130B700FF30AB00FB2123
:10081000AB0B0B2C0800B20A072CAC01F3116400DF
:100820008C1A282C0C18152C0F2C67308F002E30AA
:100830008E000C10AC0A731D1F2C2030202C703041
:100840002C06031D0F2CF3150800A4018C1E0800B4
:100850001A08A4009818372C18193A2C0D302406C1
:100860000319362C6D1D362C2408E42108001812BB
:10087000181608001A080800613024020318412CD9
:1008800008007B302402031C462C08002030A40200
:100890000800AA01EA240D30240603195D2C20303B
:1008A0002406031D5D2C742CEA240D302406031944
:1008B000772C203024060319772C30302402031CB7
:1008C000742C3A3024020318742C3030A4020930FE
:1008D000AB002A08AA070318742CAB0B6A2C240857
:1008E000AA070318742C542C0301031408002A08C7
:1008F000031008000A3051228C1E802C1A087A2C12
:100900009818852C1819882C080018121816080039
:100910001A080800AA00AB00F030AB050310AB0CBE
:10092000AB0CAB0CAB0C00308A002B084820E42148
:100930000F302A054820E421080024308400FB23DE
:100940000800AC00693084002C0884070008A80067
:10095000253084002C0884072808800008007512C0
:1009600000308A00AB0125302B07840000080319F2
:10097000C22C80030008031DC22C2B084520F40460
:100980002B08A124AB0A02302B06031DB32C080050
:10099000B2010D24F319E72C2408083A0319D12CCD
:1009A000D72C030132060319C92CB203C92C240821
:1009B000B700FB21B20A0A3024060319E72C0330E2
:1009C00024060319E72C7C303206031DC92CB7011D
:1009D000FB2108001122A400B20AF3183C240800ED
:1009E0000408A9000630AB000008AC0020302C063B
:1009F0000319FC2C2C08E421AB030319012D840AF4
:100A0000F42C2D30E421840A0F300005AC000A30AC
:100A10002C02031C0F2D3130E4210A30AC0230309F
:100A20002C07E4212908840008008C1E0800F31418
:100A3000C824F72603181E2D0230A22EAC00053064
:100A40008A002C088207672D872D9A2D582DCA2DD4
:100A5000C82DCC2DCF2DD52DE02DEF2DD22DF12D64
:100A6000DC2D652DED2DC12D0000852D912E942EB0
:100A7000962E8B2E8E2E0000982E9B2E9E2E542D61
:100A8000412D49240318A22EAC000D302406031D6D
:100A9000A22EC9302C020318A22E00302C060319F6
:100AA000A22E2C08EB00A42E1D30CC23CF27A42E81
:100AB00061308400B126030104060319652D0D3051
:100AC0002406031D652DEC17A42EEC13A22E492439
:100AD0000318A22EAC000D302406031DA22E3D30BB
:100AE0002C020318A22E00302C060319822D0F3081
:100AF0002C02031C0310AC0D2C0DE9000301A124F2
:100B0000EC15A42EEC11E901A42EE923A42E0E303D
:100B1000CC236C1F942D6D1C972D7A24F514751021
:100B2000F3100430CC2308000B30CC23A22E0A3063
:100B3000CC23A22E4530A90029088400B126030148
:100B400004060319C12D5A302906031DAC2D0D30A2
:100B500024060319C42DC12D0D3024060319C42DFC
:100B600020302406031DC12DEA2456302406031D1F
:100B7000C12DEA2420302406031DC12D0730A9070A
:100B80009C2D6D10E801A22E6D142908E800A42EFA
:100B9000EC16A42EEC12A42E6C166C11A42E6C155F
:100BA0006C12A42E6C126C11A42E3E308400B1265F
:100BB00003010406031DDE2D6C13A22E6C17A42E58
:100BC0006430AB00F310EA2424089E27AB0A240803
:100BD000003A031DE32DED14A42EED10A42E902752
:100BE000A42E6D19F62D1230CC23F82D1130CC2304
:100BF0001E30CC2308308A006B08002003308A00A6
:100C00000E30CC231630CC23ED1E092E1730CC230A
:100C1000102E6D1F0E2E1B30CC23102E1C30CC231B
:100C20000E30CC23ED191C2E6D1A192E1330CC2347
:100C30001F2E1430CC231F2E1530CC231F2E0E3028
:100C4000CC230630CC236C1A292E6C192B2E19308C
:100C50002C2E07302C2E1830CC23EC1A322E0930D3
:100C6000CC23342E0830CC23EC1D442E1030CC2362
:100C70006908AC0008308A000310AC0C2C0C002072
:100C800003308A000E30452E0F30CC230A30CC239F
:100C90006D184D2E0E30CC235F2E45308400F0248D
:100CA0000730840704086802031C5D2E2030E4210D
:100CB0005630E4212030E4214F2E0E30CC230B306F
:100CC000CC236C1F662E3E308400F0240E30CC23E3
:100CD0000C30CC23EC1F6F2E61308400F0240E30DA
:100CE000CC230D30CC23ED1C882E6430AB002B08B8
:100CF000831203178D00831603170C148312031736
:100D00000C08831203130319A42EE421AB0A772ED7
:100D10000E30CC23A62E6D16ED11A42EED156D12FE
:100D2000A42EED116D12A42E6D15A42E6D11A42EFE
:100D3000ED166D13A42E6D17ED12A42EED176D1385
:100D4000ED12A42E0530A52E0330CC230130CC2388
:100D50007A24F31008006C16EC166D154030EB0089
:100D600008000408A8000730B10020308000840A81
:100D7000B10BB52E28088400B101EA242D302406D9
:100D80000319DB2E0D3024060319D52E203024063E
:100D90000319D52E28083107840024088000B10AE1
:100DA0003108073A031DBD2EF52E063028078400B2
:100DB00030308000F22E49240318F52E303EAC006E
:100DC00040302C020318F52E0630280784002C082A
:100DD00080000D3024060319F22E2030240603195A
:100DE000F22EF52E280884000800840108008312E2
:100DF00003170C308F00DA308D0083120313B20119
:100E0000EA242627AC0024060319192F2C082402F3
:100E1000031C172F013033272627AC0000302C0687
:100E20000319172F01303B272C083327012F0310FC
:100E30000800023033272627AC00FF302C06031DA4
:100E4000002F0130332726270314080083160317C9
:100E50008C170C14000000008C13831203170C086D
:100E6000831203130800831203178D0703188F0AD8
:100E7000831203130800831203178D02031C8F03D0
:100E80008312031308008C1E0800C824F319622F74
:100E9000033024060319622F0D30E4210A30E421C7
:100EA000B2012421F310EA24033024060319622F2F
:100EB0000301240603195F2F24088221532F6D217B
:100EC000C0210800C021F51075147A240130CC230C
:100ED0000800B201BB011122A4003C242C302406DE
:100EE000031D742F3B080800B20A2408BB076B2FB0
:100EF000AB013E3084002B08831203178D0083164C
:100F000003178C010C14831203170C0883120313AC
:100F100080002F302B0603190800840AAB0A7B2FB0
:100F2000AB013E3084008312031300089E272F304C
:100F30002B0603190800840AAB0A932F0D128312A3
:100F400003178C00831203132B08831203178D00E1
:100F5000831603170C158B1355308D00AA308D00A6
:100F60008C140C11831203130D1EB42F0D128B174A
:100F7000080064000C18BD2FCB2F67308F002E3077
:100F80008E000C10A70AEF302706031DCB2F751615
:100F9000A7010314080003108C1A031408007B2017
:100FA0005F2164002524203024060319DC2F033040
:100FB00024060319DE2FD12F6B20D12FC02108006A
:100FC0009D2402249120AA20F517851EED2F0030C4
:100FD000CC230130CC237514F02F73156C126C11D7
:100FE000640075181525F5184327751AAF24741871
:100FF000D720F51B8C22F51A5923751BF222F02FEE
:10100000AC00AB01A801A90108308A002B082420FC
:10101000003A031923282C02031C1128AC00A90A4A
:10102000042803012906031916281828281C20283B
:1010300001308A00281430302907E42108308A0062
:10104000A901AB0A04280800820764340A34013479
:1010500000340D340A3443346F346D346D346134EC
:101060006E34643473342034613472346534203423
:101070004334613473346534203449346E3473340A
:1010800065346E3473346934743469347634653459
:101090000D340A34553473346534203442346134A9
:1010A00063346B34733470346134633465342034A6
:1010B0004B34653479342034283442345334293461
:1010C000203466346F347234203443346F347234D5
:1010D000723465346334743469346F346E340D346F
:1010E0000A345534733465342034743468346534C8
:1010F00020344434493453345034203463346F340E
:101100006D346D3461346E346434203474346F342F
:10111000203464346934733470346C346134793419
:10112000203461346C346C3420346F347034743453
:1011300069346F346E3473340D340A3449346E3488
:10114000733465347234743420344A3475346D34F5
:1011500070346534723420344A3434342034613489
:101160006E346434203443346F346E346E346534FA
:101170006334743420344734503453342034663468
:101180006F34723420344134503452345334203468
:101190004F347034653472346134743469346F346C
:1011A0006E340D340A34523465346D346F34763411
:1011B000653420344A3475346D3470346534723497
:1011C00020344A343434203461346E34643420346E
:1011D00043346F346E346E34653463347434203485
:1011E00074346F3420345434653472346D3469345B
:1011F0006E3461346C34203466346F34723420348D
:1012000043346F346D346D3461346E34643420345F
:1012100049346E34743465347234703472346534E5
:101220007434653472340D340A340D340A34433462
:101230006F346D346D3461346E34643473342034FF
:10124000283477346934743468342034653478341D
:1012500061346D3470346C34653429343A3420345C
:101260000D340A344D345934433441344C344C3405
:10127000203428346D347934633461346C346C3404
:1012800020347734623438347734673461342D3421
:10129000323429340D340A345534503450345234F5
:1012A0004F3454344F342034283475346E34703411
:1012B00072346F3474346F34203477346234383499
:1012C0007734673461342D34313434342034763417
:1012D00020347734623438347734673461342D34D1
:1012E0003134293420342D342034333420346434E0
:1012F000693467346934733420346D34613478343C
:101300000D340A344234543445345834543420347F
:10131000283462347434653478347434203442347C
:101320006F34623429342D34313430343034203445
:101330006334683461347234733420346D3461340E
:1013400078340D340A3442344534413443344F3414
:101350004E342034283462346534613463346F345D
:101360006E34203465347634653472347934203404
:101370006E3429342D3420346E343D3430342034EE
:101380006934733420346F34663466342034613405
:101390006E346434203431343C346E343C3436346E
:1013A000303420346D3469346E3473340D340A347F
:1013B0004D344F344E34693474346F3472342034C5
:1013C00028346D346F346E34203461346C346C34B2
:1013D0002C346D346F346E3420346D3465342C34D9
:1013E00020346F34723420346D346F346E342034D2
:1013F0006F346634663429340D340A344434493445
:1014000047344934703465346134743420342834BA
:10141000643469346734693420346F346E34203472
:101420006F3472342034643469346734693420345E
:101430006F346634663429340D340A344D345934EB
:1014400041344C34493441345334203428346D34DD
:10145000793461346C3469346134733420345234F7
:1014600045344C344134593429340D340A34503421
:10147000453452344D3420342834503445345234B9
:101480004D3429340D340A344534433448344F3410
:10149000203428346534633468346F3420346F3436
:1014A0006E3420346F3472342034653463346834DD
:1014B0006F3420346F346634663429340D340A3482
:1014C0004734503453342034283467347034733400
:1014D00020342434473450344734473441342034A2
:1014E0006F347234203467347034733420342434CD
:1014F0004734503447344C344C3420346F347234D5
:1015000020346734703473342034243447345034F6
:1015100052344D34433429340D340A345434523463
:1015200061346334653420342834743472342034A4
:1015300078346D346934743420346F347234203428
:101540007434723420347234633476342934203461
:101550002D34203446346F3472342034643465348E
:10156000623475346734673469346E3467342034D8
:101570006F346E346C3479340D340A345434583446
:10158000443445344C344134593420342834743490
:101590007834643465346C346134793420346E3496
:1015A000203430343C346E343C34323430343134D2
:1015B00020346E3420346934733420346E347534FE
:1015C0006D3462346534723420346F3466342034C0
:1015D000643465346C3461347934203466346C346A
:1015E000613467347334203474346F34203473348A
:1015F00065346E34643429340D340A344334413450
:101600004C34493442345234413454344534203417
:101610002834433461346C34693462347234613454
:101620007434653420344D346F346434653420347C
:101630002D342034543465347334743469346E3446
:10164000673420344F346E346C34793429340D349B
:101650000A340D340A3400344B0B800B880B8A0B90
:101660008F0BB50BB90BC20BC80BD80BE90BF20BE8
:10167000FA0B030C0A0C0D0C1A0C2B0C370C440C37
:101680004E0C580C640C690C700C750C7B0C950C92
:101690009C0CA30CD10C0D340A345734423438342A
:1016A00057344734413420344D344F344434453476
:1016B0004D344C34453453345334203454344E3444
:1016C0004334203420345634203431342E343034F2
:1016D00038340D340A345434793470346534203459
:1016E000483445344C345034203466346F347234CA
:1016F000203449346E3466346F340D340A34003487
:101700000D340A3463346D3464343A342034003494
:101710003F3400340D340A344F344B3400340D342C
:101720000A342A342A342A342034203443346F349F
:101730006E347634653472347334653420344D3409
:101740006F34643465342C342034633474346C3432
:1017500020344334203474346F34203445347834A6
:10176000693474340D340A3400340D340A343F348F
:1017700000344D344F344E34693474346F34723421
:101780002034003441344C344C340D340A340034A9
:1017900044344934473449347034653461347434E2
:1017A0006534723420344F344E340D340A340034EE
:1017B00044344934473449347034653461347434C2
:1017C0006534723420344F34463446340D340A3490
:1017D000003455344E34503452344F3454344F3432
:1017E000203400344D345934433441344C344C3477
:1017F000203400344D34593441344C34493441346C
:10180000533420340034423454344534583454343E
:10181000203400340D340A34003442344534413429
:1018200043344F344E3420344F34663466340D34F0
:101830000A34003442344534413443344F344E3456
:1018400020344F346E3420344534563445345234C9
:101850005934203400340D340A3445344334483488
:101860004F3420344F344E340D340A3400340D34A8
:101870000A344534433448344F3420344F344634EA
:1018800046340D340A3400345434523461346334F1
:10189000653420344F3446344634003454345234A2
:1018A0006134633465342034523443345634003464
:1018B0005434523461346334653420342034583421
:1018C0004D34493454340034473450345334203484
:1018D000003424344734503452344D3443340034CB
:1018E0004D3445340D340A3400344F3446344634D4
:1018F0000D340A340034573461347434633468343A
:10190000203444346F3467342034543469346D34B3
:101910006534723420344634613469346C3475343F
:10192000723465340D340A3400342434473450346E
:1019300047344C344C340034243447345034473426
:10194000473441340034433461346C346934623494
:10195000723461347434653420344D346F346434FB
:1019600065342E34203453345034203474346F347E
:10197000203474346F34673467346C3465343B34EA
:101980002034633474346C3420344334203474345D
:101990006F34203445347834693474340D340A3467
:1019A000003454345834443445344C34413459347C
:1019B0002034003442342C3445341A344134003459
:1019C000433400344F3400344E3400342034003477
:1019D0004534003456340034453400345234003435
:1019E0005934003420340034FF340034543400348B
:1019F0004534003458340034543400340D34043445
:101A0000FF340F3420340034FF3409344334263497
:101A1000413412344C3400344934003442340034FC
:101A200052340034413400345434003445340034EA
:101A3000FF341C344F3400344E34003456340034F8
:101A400045340034523400345334003445340034C7
:101A50000D340034FF34013444342234493400342A
:101A60004734163449340034203400344F340034C1
:101A700046340834463400340D340034FF34043422
:101A80004E3400340D340034FF3405345334003404
:101A9000503400340D340034FF340C3445341A34DF
:101AA00043340034483400344F340034203400349C
:101AB0004F34003446340834463400340D34003496
:101AC000FF3415344E3400340D340034FF341434F4
:101AD0004734243450340034533400342034003438
:101AE00024340034473400345034003447340E3446
:101AF0004734063441340034FF341B344C34003452
:101B00004C340034FF341A34523400344D34003431
:101B100043340034FF34193448340C344534003431
:101B20004C340034503400340D340034FF3412345B
:101B30004D344A344F3424344E340034203400348D
:101B4000413408344C3400344C340034FF3406340F
:101B50004D34063445340034FF3407344F340034F8
:101B600046340834463400340D340034FF340B342A
:101B70004E3400340D340034FF340734593400340B
:101B8000413412344C34003449340034413400348C
:101B9000533400340D340434FF340E342034003414
:101BA000FF34033443340034413400344C340034C3
:101BB0004C3400340D340434FF340D3420340034FC
:101BC000FF34083450340C3445340034523400347B
:101BD0004D3400340D340034FF340A345434363478
:101BE00052342434203400344F340A344634003420
:101BF000463400340D340034FF34133452340A3484
:101C000043340034563400340D340034FF34163479
:101C1000583400344D3400344934003454340034E2
:101C20000D340034FF341734583400344434003455
:101C3000453400344C3400344134003459340034D9
:101C400020340034FF341D34553400344E34003415
:101C500050340034523400344F340034543400349F
:101C60004F3400340D340434FF3410342034003445
:041C7000FF34023407
:02400E000A3F67
:02401000FC3F73
:00000001FF
